:1000000038C09EC150C050C04EC04DC04CC04BC047
:100010004AC049C09FC147C046C045C067C143C030
:1000200042C041C040C053EF6E310000000053EFAA
:100030006E35000000004578697400000000200A59
:1000400052756E6E696E672054696D653A0A006874
:1000500028486F757229200068284D696E290A00AA
:100060006828486F757229200068284D696E290A32
:10007000000011241FBECFE5D4E0DEBFCDBF10E0ED
:10008000A0E6B0E0E0E2F9E102C005900D92A036F2
:10009000B107D9F713E0A0E6B0E001C01D92A43982
:1000A000B107E1F784C1ACCF1F920F920FB60F9248
:1000B00011242F933F934F935F936F937F938F936D
:1000C0009F93AF93BF93EF93FF9380917B0388231C
:1000D00029F080917B03815080937B0320919003D2
:1000E0002223C9F480917E038F5F80937E038091E9
:1000F0007E03843658F080917C0390917D038C5A66
:1001000091400CF4919820937E0305C080917E036A
:10011000823309F4919A809170038F5F809370030A
:10012000809170038436E8F01092700380918A0306
:100130008F5F80938A0380918A038C3390F01092B2
:100140008A0380917A038F5F80937A0380917A0388
:100150008C3338F010927A03809193038F5F8093F1
:10016000930390918703109287039B9913C090FF8C
:100170000BC0809164008F5F809364008091640065
:10018000882329F48FEF01C081E08093640081E02F
:10019000809387039A9915C091FF0BC080918903C2
:1001A0008F5F8093890380918903882329F48FEFDF
:1001B00001C081E0809389038091870382608093EE
:1001C0008703999915C092FF0BC0809175038F5FCB
:1001D0008093750380917503882329F48FEF01C004
:1001E00081E0809375038091870384608093870307
:1001F000989932C0809180038F5F809380038091B3
:100200008003882319F48FEF80938003809180030B
:100210008431E0F080918803885F80938803809127
:100220008803803B18F088EA8093880380918803D4
:100230009927382F2227809188039927282B392B3B
:10024000B9018BE0A1D981E080938003809187037D
:1002500088608093870302C010928003B09931C0F8
:1002600080918B038F5F80938B0380918B03882316
:1002700019F48FEF80938B0380918B038431D8F036
:100280008091880388508093880380918803883FF9
:1002900010F010928803809188039927382F222725
:1002A000809188039927282B392BB9018BE06CD9D1
:1002B00081E080938B038091870380618093870323
:1002C00002C010928B038EEC86B9FF91EF91BF9123
:1002D000AF919F918F917F916F915F914F913F91DE
:1002E0002F910F900FBE0F901F9018951F920F9295
:1002F0000FB60F9211242F933F938F939F9384B146
:10030000282F332785B1992783709070982F8827DD
:1003100090937D0380937C0380917C0390917D0377
:10032000822B932B90937D0380937C0337989F912E
:100330008F913F912F910F900FBE0F901F901895A6
:100340001F920F920FB60F9211240F900FBE0F90B5
:100350001F9018951F920F920FB60F9211242F9392
:100360008F939F93EF93FF9380918E0390918F03D0
:10037000FC01EA59FF4F2FB12083019690938F0320
:1003800080938E0380918E0390918F0380509240D2
:1003900014F06F9802C08FEF8FB9FF91EF919F918A
:1003A0008F912F910F900FBE0F901F901895CFE552
:1003B000D4E0DEBFCDBF8DE088BB8EE287BB8FE08F
:1003C00085BB80E184BBC1E0C2BB88EF81BB04B6C2
:1003D00003FE02C08C2FE2D714BE9B9B09C0C093C2
:1003E000900310BC98E199B980E28BB99AB904C026
:1003F00010929003899A919AA89588E181BD8FE126
:1004000081BD85EC87B9479A8FE085BD8DE483BDBA
:1004100089B7806889BF83E885BF8BB780648BBF4D
:100420001092870310927D0310927C031092710347
:10043000789480917C0390917D038A59914044F493
:10044000889580917C0390917D038A599140C4F3F3
:10045000AC9A82E380937B038CE033D8809388034B
:1004600080918803992787709070079719F488E422
:100470008093880381E025D8992790938603809301
:10048000850383E01ED89927982F882790936702C9
:100490008093660282E015D8282F33278091660268
:1004A00090916702822B932B909367028093660250
:1004B00086E007D89927AA27BB27DC019927882738
:1004C0008093760390937703A0937803B093790396
:1004D00085E0F7D79927AA27BB272227382F492F4E
:1004E0005A2F8091760390917703A0917803B09171
:1004F0007903822B932BA42BB52B809376039093B7
:100500007703A0937803B093790384E0DAD7282F98
:100510003327442755278091760390917703A09144
:100520007803B0917903822B932BA42BB52B809366
:10053000760390937703A0937803B09379038BE0CD
:10054000C0D79927AA27BB27B82FAA27992788277A
:1005500080936A0390936B03A0936C03B0936D0335
:100560008AE0AFD79927AA27BB27AC0133272227D8
:1005700080916A0390916B03A0916C03B0916D031D
:10058000822B932BA42BB52B80936A0390936B0340
:10059000A0936C03B0936D0389E093D79927AA27A2
:1005A000BB272227382F492F5A2F80916A03909119
:1005B0006B03A0916C03B0916D03822B932BA42B42
:1005C000B52B80936A0390936B03A0936C03B09355
:1005D0006D0388E076D7282F33274427552780914D
:1005E0006A0390916B03A0916C03B0916D03822B11
:1005F000932BA42BB52B80936A0390936B03A0934A
:100600006C03B0936D031092700310928A038EE016
:1006100058D780937A038DE054D7809393038091C9
:100620007A038F3F21F410927A0310929303809102
:1006300090038823D9F08EE390E013D9809193033F
:10064000FBD88FE490E00DD980917A03F5D888E546
:1006500090E007D98FE035D7EFD880E690E001D958
:1006600080E12FD7E9D889E690E0FBD88091870315
:1006700081FF04C0109267021092660280917B0392
:10068000882329F0889580917B038823D9F781E01E
:1006900026D18F3F31F4C19A61E083E01AD781E01F
:1006A0007DD6C19AA89560E081E013D760D18823F8
:1006B00029F061E082E00DD781E070D68FEF9FEFE7
:1006C00050D29093690280936802892B29F461E0EB
:1006D000862FFFD681E062D68091850390918603B4
:1006E000892B31F481E090E0909386038093850319
:1006F000809185039091860334D260918602809127
:1007000087029927AA27BB272227382F492F5A2F3C
:10071000260F311D411D511D809188029927AA275E
:10072000BB27DC0199278827280F391F4A1F5B1F29
:10073000809189029927AA27BB27B82FAA27992732
:100740008827280F391F4A1F5B1F80916A039091E9
:100750006B03A0916C03B0916D0382179307A407FC
:10076000B50751F081E090E0909386038093850374
:100770001092670210926602D2D6209185033091C2
:10078000860380916802909169028217930730F482
:1007900081E090E090938603809385038BD08091D5
:1007A000760390917703A0917803B09179039C012F
:1007B000AD0160916602709167028091850390910E
:1007C000860370D2C82F76D0C7FF05C0C19561E0FF
:1007D0008C2F7FD636C0C130B9F580916400853644
:1007E00080F180917C0390917D038D5F914014F0A6
:1007F00060E025C080917C0390917D03895E9140EB
:1008000014F060E019C080917C0390917D03855DB8
:10081000914014F060E04BC080917C0390917D0387
:10082000815C91400CF042C080917C0390917D03EB
:100830008D5A91401CF06C2F82E03AC06C2F83E0FF
:1008400037C080E0ABD52AC0C330D9F4809189038A
:10085000853618F081E090E019C0809189038A31D3
:10086000C8F0809185039091860301979093860349
:1008700080938503892B71F48091680290916902BD
:1008800005C080918503909186030196909386031D
:1008900080938503109267021092660280917C0318
:1008A00090917D038A5991400CF067CF61E081E01F
:1008B00010D663CF7894A895889588958091870302
:1008C000992787709070892BB1F7889588958091CA
:1008D0008703992787709070892B69F708951F9374
:1008E000CF93182F882311F08EE501C082E58DB9D2
:1008F000C29AC0E064D7CF5FC431E0F3C29840E051
:1009000050E060E070E080E0F3D6C82F8130B9F0AD
:100910008F3FA9F080919003882321F08C2F8CD7F2
:1009200080E286D78895889540E050E060E070E0EE
:1009300080E0DED6C82F813011F08F3F59F7C130EB
:1009400049F440E050E060E070E081E0D1D6C82F8B
:100950008130B9F3C29A112311F08CE501C080E512
:100960008DB9709A8C2F9927CF911F910895EF928E
:10097000FF920F931F93CF93DF936EEB71E080E0B4
:1009800090E024D620917202809173029927D82F8B
:10099000CC27C20FD11D7E010027112749E0EE0CA4
:1009A000FF1C001F111F4A95D1F7C801B7010ED6D1
:1009B00020917502809176029927982F8827820FBF
:1009C000911D8050924019F082E090E0C3C0809168
:1009D00077028093650080917802FE01E80FF11D97
:1009E000809179029927982F8827E80FF91FF093B3
:1009F0008D03E0938C0320917B0280917C029927E8
:100A0000782F6627620F711D709392036093910394
:100A100020918002809181029927582F4427420F0C
:100A2000511D4115510519F481E090E093C080916A
:100A30007A029927849FE001859FD00D949FD00D65
:100A40001124CE018E0F9F1F909374038093730324
:100A5000AB01A4E056954795AA95E1F76F707070C9
:100A6000672B11F04F5F5F4FAA27BB27EA01EE27E4
:100A7000FF278C0F9D1FAE1FBF1F809360009093B8
:100A80006100A0936200B093630020917D02809189
:100A90007E029927AA27BB27FA2FE92FD82FCC2728
:100AA000C20FD11DE11DF11D2097E105F10581F572
:100AB000D801C7018096A11DB11DBC01CD0186D50D
:100AC00020916A0280916B029927AA27BB27FA2FEF
:100AD000E92FD82FCC27C20FD11DE11DF11D809128
:100AE0006C029927AA27BB27DC0199278827C80F02
:100AF000D91FEA1FFB1F80916D029927AA27BB27E8
:100B0000B82FAA2799278827C80FD91FEA1FFB1FCC
:100B100080918C0390918D03AA27BB27C81BD90B0A
:100B2000EA0BFB0B80916500282F332744275527BC
:100B3000BE01CF01D3D6FA01E901C050D041E04057
:100B4000F04020F081E08093720302C010927203A3
:100B500080E090E0DF91CF911F910F91FF90EF9097
:100B600008954F925F926F927F928F929F92BF9261
:100B7000CF92DF92EF92FF920F931F93CF934C018E
:100B80006624772480917303909174037C0100277D
:100B9000112779E0EE0CFF1C001F111F7A95D1F789
:100BA000230180919103909192036816790608F0D1
:100BB00069C0C801B7014ED5882309F063C0B82EBB
:100BC000C0E06AE6C62E62E0D62EF9D5D6018D9336
:100BD0006D01CF5FC032C8F390916A02992369F129
:100BE00080918402882321F4809185028823F1F08A
:100BF000953EE1F080917502992788719070892B5C
:100C0000A9F4809172028D3489F480917302803549
:100C100069F480917402833349F40894611C711C57
:100C20000894810891088114910439F00894411CBA
:100C3000511CB394BFE0BB1518F6B394EFE0EB156D
:100C400048F0C0E0BCD5CF5FC032E0F3B394FFE022
:100C5000FB15B8F73BD580916A02882399F081147F
:100C6000910481F080E092E0A0E0B0E0E80EF91E8F
:100C70000A1F1B1F809191039091920348165906F9
:100C800008F497CFC301CF911F910F91FF90EF9080
:100C9000DF90CF90BF909F908F907F906F905F90EC
:100CA0004F9008954F925F926F927F928F929F9292
:100CB000AF92BF92CF92DF92EF92FF920F931F936A
:100CC000CF93DF938C01EB0169017A014ADF0817AA
:100CD000190719F08FEF9FEF3EC220918602809195
:100CE00087029927AA27BB274427582F692F7A2FD5
:100CF000420F511D611D711D809188029927AA27FD
:100D0000BB27DC0199278827480F591F6A1F7B1FC3
:100D1000809189029927AA27BB27B82FAA2799274C
:100D20008827480F591F6A1F7B1F40936A035093FF
:100D30006B0360936C0370936D032097D1F0D09395
:100D40006702C0936602C0927603D0927703E09266
:100D50007803F092790309E0CC0CDD1CEE1CFF1C3B
:100D60000A95D1F760906A0370906B036C187D0848
:100D700022C020918402809185029927982F88278C
:100D8000820F911D9093670280936602DB01CA0176
:100D9000C9E0B695A79597958795CA95D1F78093A1
:100DA000760390937703A0937803B09379035170FF
:100DB000607070703A0180916602909167022FEF27
:100DC0008F3F920709F473C18230910530F46FC1EF
:100DD000899399938883998318C0CAE6D2E0AA249C
:100DE000BB24899399938E0122964AD2D8018D9380
:100DF0009C93C2D1BFEF8F3F9B0751F30894A11C76
:100E0000B11CE0E4AE16B10460F380916A029091E7
:100E10006B02909367028093660240906C02509040
:100E20006D02CEE6D2E01092640010928903109217
:100E3000750320916500822E9924AA27BB2702976B
:100E4000A109B109332744275527BC01CD0127D576
:100E50006B017C018091600090916100A091620023
:100E6000B0916300C80ED91EEA1EFB1EB9E0CC0C7F
:100E7000DD1CEE1CFF1CBA95D1F78895889584E699
:100E800080937B038091760390917703A091780300
:100E9000B0917903181619061A061B060CF0FAC051
:100EA000C701B601D7D3882309F001C1F8948FEFA9
:100EB00082D4AA24BB249FB18FEF8FB9829909C035
:100EC000A89584E680937B0378948895F894829B18
:100ED000F7CF97FF02C0979A01C09798949A939A78
:100EE000990F9398949886E097FF02C0979A01C053
:100EF0009798939A990F9398815087FFF5CF08940C
:100F0000A11CB11CF0E0AF16F2E0BF06A0F278948D
:100F1000DDD38091760390917703A0917803B0910F
:100F200079030197A109B109809376039093770320
:100F3000A0937803B09379030894810891088114F1
:100F4000910451F180E092E0A0E0B0E0C80ED91E1B
:100F5000EA1EFB1E80919003882309F472C091E081
:100F60008916910409F06DC000917C0310917D03F6
:100F7000812F992761D4802F5FD480E259D480914A
:100F8000660290916702892F992756D48091660254
:100F900053D48AE04DD455C0809166029091670287
:100FA000019690936702809366024816590600F5F1
:100FB000A3E0CA36DA0748F48991999190936702C1
:100FC000809366024990599006C0D6D090936702EC
:100FD00080936602240180916602909167028230BC
:100FE000910518F08F5F9F4F19F46624772452C043
:100FF0008091660290916702AA27BB270297A109F8
:10100000B10910916500212F332744275527BC01D2
:10101000CD0145D46B017C0180916000909161000D
:10102000A0916200B0916300C80ED91EEA1EFB1E9B
:10103000E9E0CC0CDD1CEE1CFF1CEA95D1F7812EFB
:10104000992489D110917B03112351F4809171036C
:10105000181684F181E0809371031093890347C0CF
:1010600080916400833070F580917503833090F532
:10107000809189038330B0F5809176039091770356
:10108000A0917803B0917903181619061A061B0669
:101090000CF406CF10927103C30101978F5F91404A
:1010A00008F055C0C701B601D5D2882319F18EEFDB
:1010B0009FEF51C061E0862F0CD210937103109303
:1010C00075030DC060E081E004D21092710381E0ED
:1010D00090E041C060E081E0FCD11092710382E0B9
:1010E00090E039C060E081E0F4D11092710383E0B8
:1010F00090E031C0F8948FEF5ED3AA24BB242FB1C7
:101100008FEF8FB9C301089461087108892BA9F08A
:10111000829905C0A8957894F894829BFBCF949A05
:1011200087E027FF02C0979A01C09798939A220FF1
:1011300093989498815087FFF4CF0894A11CB11C18
:10114000F0E0AF16F2E0BF06D0F27894BFD28895F7
:10115000889580E090E0DF91CF911F910F91FF90F3
:10116000EF90DF90CF90BF90AF909F908F907F9047
:101170006F905F904F900895CF92DF92EF92FF9221
:101180000F931F93CF93DF936C0180917203609153
:101190008C0370918D03960144275527882309F00D
:1011A0004CC07B0100271127B9E0EE0CFF1C001F8B
:1011B000111FBA95D1F7E20EF31E041F151FC601C9
:1011C00096958795AA27BB27E80EF91E0A1F1B1FB5
:1011D000D801C7019170A070B0708F5F9140A0409E
:1011E000B04091F4C801B70159D0EC01D070089417
:1011F000E11CF11C011D111DC801B7014FD0982F32
:101200008827C82BD92B04C0C801B70147D0EC01EF
:10121000C0FE07C06E01E4E0D694C794EA95E1F7FA
:1012200006C07FEFC72E7FE0D72ECC22DD2288EFCD
:10123000C8168FE0D806D0F016C0CB01AA27BB276E
:10124000BA2FA92F982F8827820F931FA41FB51F8D
:10125000880F991FAA1FBB1FBC01CD011FD06C01B5
:10126000885F9F4F18F05FEFC52ED52EC601DF9126
:10127000CF911F910F91FF90EF90DF90CF90089545
:10128000CF93DF93EC01CE0177DF2196C817D90702
:10129000D1F32197CE01DF91CF910895CF92DF92C4
:1012A000EF92FF920F931F93CF93DF937B018C01FB
:1012B0008FEFC82E81E0D82ECE20DF2080E09EEF79
:1012C000AFEFBFEFE822F9220A231B2380918103AD
:1012D00090918203A0918303B0918403E816F906EC
:1012E0000A071B07E9F0C801B701B4D1882319F038
:1012F00020E030E026C0C6E6D0E092E0C636D9074E
:1013000030F45DD28993A2E0C636DA07D0F3DED19D
:10131000E0928103F092820300938303109384038D
:10132000F601EA59FF4F8081282F3327E7E6F0E0E6
:10133000CE0EDF1ED6018C919927982F8827282B57
:10134000392BC901DF91CF911F910F91FF90EF9041
:10135000DF90CF90089580917C0390917D038C570E
:101360009140BCF4C29A61E084E0B3D0F8948091DB
:101370009303882361F060917A0380E191D06091BA
:1013800093038FE08DD010927A031092930380E044
:1013900005D080917C0390917D0308951F93182FB1
:1013A000F894C29AC19860E170E080E0EDD011231A
:1013B00009F072C0609188038CE072D0609185035F
:1013C00081E06ED06091660282E06AD08091660210
:1013D00090916702892F9927682F83E061D06091EF
:1013E000760384E05DD08091760390917703A0919D
:1013F0007803B0917903892F9A2FAB2FBB27A7FDD4
:10140000BA95682F85E04CD0809176039091770350
:10141000A0917803B0917903CD01BB2797FDB095DA
:10142000AB2F682F86E03CD060916A0388E038D00B
:1014300080916A0390916B03A0916C03B0916D034E
:10144000892F9A2FAB2FBB27682F89E029D0809155
:101450006A0390916B03A0916C03B0916D03CD0171
:10146000AA27BB27682F8AE01BD080916A0390913E
:101470006B03A0916C03B0916D038B2F9927AA2762
:10148000BB27682F8BE00CD060917A038EE008D0E8
:10149000609193038DE004D0AC98A8958895FCCF1B
:1014A0001F93CF93C82F162F0CD0811739F0E199D5
:1014B000FECF1FBACEBB1DBBE29AE19ACF911F911E
:1014C0000895E199FECF1FBA8EBBE09A8DB399279C
:1014D00008951F93CF93C82F162FF89420D0789497
:1014E000CC23B9F0112319F08EE290E002C086E21D
:1014F00090E033D083E18895815087FFFCCF86E36D
:1015000090E02BD085E08895815087FFFCCFC150BB
:1015100049F786E390E021D0CF911F91089564E0D0
:1015200070E080E031D090D060E070E080E02CD0BE
:10153000829BFECF809188039927382F22278091A4
:1015400088039927282B392BB9018BE01DD060E740
:1015500077E983E019D078D0089540E0FC01019646
:101560002491949A30E027FF02C0979A01C097987F
:10157000939A220F939894983F5F3830A0F3979AEC
:101580004F5F483058F30895FF920F931F93F82E42
:101590008B01959882E00CD08F2D0AD0812F99274E
:1015A00007D0802F05D0959A1F910F91FF90089535
:1015B00097E087FF02C0979A01C09798969A880F84
:1015C0009698915097FFF5CF979A0895CF92DF9212
:1015D000EF92FF920F931F93CF93DF937B018C01C8
:1015E000DC01CB0180709E7FBC01CD0133D088230C
:1015F00011F5BFEFCB2EB1E0DB2ECE20DF2000E0D7
:1016000010E00C151D0579F4CAE6D2E0AFE1EA2E30
:10161000F12CEC0EFD1ED3D089930F5F1F4FEC16FB
:10162000FD06CCF701C0CBD00F5F1F4F82E000302A
:10163000180738F34BD0DF91CF911F910F91FF9096
:10164000EF90DF90CF90089580E000008F5F8F3F94
:10165000E1F70895DF92EF92FF920F931F93CF93DC
:10166000DF937B018C01DD24C298B801A70181E1E1
:101670003FD0982F882361F4C0E0D0E0A0D0982F0D
:101680008E3F41F021968FE0C03AD807B8F305C0ED
:101690008E3F19F480E090E011C0C29A80919003CF
:1016A000882321F0892FC8D080E2C2D08895889500
:1016B000D39483E68D15C0F681E090E0DF91CF9161
:1016C0001F910F91FF90EF90DF900895CF93DF93DC
:1016D00076D075D0C0E0D0E072D08F3F29F021964F
:1016E00083E0C83ED807C0F3C29ADF91CF91089536
:1016F000AF92BF92DF92EF92FF920F931F93CF931F
:10170000DF93CDB7DEB721970FB6F894DEBF0FBEDB
:10171000CDBFD82E7A018B01AA24BB2450D0982F9C
:101720008F3F41F00894A11CB11C88EEA81683E0FD
:10173000B806A0F39F3F39F081E090E02CC0998378
:101740003ED0998126C0E0E4DE2A8D2D34D0812F51
:101750009927AA27BB272FD0C801AA27BB272BD0A0
:10176000BB27A12F902F8F2D26D08E2D24D085E939
:1017700022D0AA24BB2423D0982F8E3F51F0882357
:10178000F4F60894A11CB11CF8EEAF16F3E0BF0606
:1017900090F3892F992721960FB6F894DEBF0FBEDC
:1017A000CDBFDF91CF911F910F91FF90EF90DF9010
:1017B000BF90AF9008958FB9779BFECF08958FEFBC
:1017C0008FB9779BFECF8FB199270895779BFECF76
:1017D0000895CF93DF93DC01CB0139E0880F991F87
:1017E000AA1FBB1F3A95D1F7BC01CD0133DF24D02E
:1017F0008AE01ED0C0E0D0E0E2DF1ED0CE018F71C3
:1018000090704F9711F48AE003C0C0FF02C080E2DD
:101810000FD0219682E0C030D80774F357DFDF91F4
:10182000CF910895A8955F9BFDCF8CB1992708951E
:101830005D9BFECF8CB90895CF93C82F982F9295BA
:101840009F70892F805D8A3308F0895FF1DF9C2FBC
:101850009F70892F805D8A3308F0895FE9DFCF911F
:101860000895CF93DF93EC01FC01219684918823A6
:1018700031F0DEDFFE01219684918823D1F7DF91DC
:10188000CF910895CF93DF93EC018991882321F0C4
:10189000CFDF89918823E1F7DF91CF910895629F8F
:1018A000D001739FF001829FE00DF11D649FE00D58
:1018B000F11D929FF00D839FF00D749FF00D659FB9
:1018C000F00D9927729FB00DE11DF91F639FB00DB8
:1018D000E11DF91FBD01CF0111240895A1E21A2EC7
:1018E000AA1BBB1BFD010DC0AA1FBB1FEE1FFF1FC4
:1018F000A217B307E407F50720F0A21BB30BE40B14
:10190000F50B661F771F881F991F1A9469F760955A
:101910007095809590959B01AC01BD01CF01089514
:00000001FF
